:100000000C94D7020C94F4020C940F030C94F40299
:100010000C94F4020C94F4020C940E200C94F40250
:100020000C94F4020C94F4020C94F4020C94F40278
:100030000C94F4020C94F4020C9497200C94F402A7
:100040000C94F4020C94F4020C94F4020C94F40258
:100050000C94F4020C94F4020C94F4020C94F40248
:100060000C94F4020C94F402A007A007CC07CC0770
:1000700022084008230923094508AD08BE08BE0828
:10008000F8176A180018CA17CE170418D1170718DE
:100090001218DC176018E0171618E4171A1844181D
:1000A000E8171E184E18EE1724182E18D5170B181F
:1000B000D8170E18F31729183A185A185C18C617CB
:1000C000FC177318AF1CB51CA31CA91CBB1CC11CBE
:1000D000C71CF31DF61D2D1E401E481E531E561E26
:1000E000561E561E9E1E9E1E5B1E5E1E631E701EAC
:1000F0007D1E801E841E911E35001E001F002000E4
:100100002100220023002400250026002700AE0045
:100110002B0014001A000800150017001C0018001E
:100120000C00120013002A0029000400160007002A
:1001300009000A000B000D000E000F003300340010
:10014000E1001D001B000600190005001100100051
:100150003600370038002800E000E300E2002452B7
:1001600021522C002C0022525000510052004F000E
:10017000AA00A9000000000000000000010001002A
:1001800001000100010001000100010001002D003B
:100190002E00010001003A003B003C003D00010040
:1001A0000100010001002F00300031004C003E0032
:1001B0003F0040004100010001000100010001007A
:1001C000010001000100420043004400450001001D
:1001D0000100010001000100010001000100010017
:1001E0000100010001000100010023524A004E00FD
:1001F0004B004D002B032B0100000000000000000D
:1002000001000100010001000100010001000100E6
:1002100001000100010001000100010001000100D6
:1002200001000100010001000100010001000100C6
:1002300001000100010001000100010001000100B6
:1002400001000100010001000100010001000100A6
:100250000100010001000100010001000100010096
:100260000100010001000100235201000100010012
:10027000010001000100010050014F0100000000D9
:100280000000000001000100010001000100010068
:100290000100010001000100010001000100010056
:1002A0000100010001000100010001000100010046
:1002B0000100010001000100010001000100010036
:1002C0000100010001000100010001000100010026
:1002D0000100010001000100010001000100010016
:1002E0000100010001000100010001000100010006
:1002F0000100010001000100037C027C1D011C01C2
:1003000000000000000000000100010001000100E9
:1003100001000100010001000100010001000100D5
:1003200001000100010001000100010001000100C5
:1003300001000100010001000100010001000100B5
:1003400001000100010001000100010001000100A5
:100350000100010001000100010001000100010095
:100360000100010001000100010001000100010085
:100370000100010001000100010001000100010075
:10038000DB00DC00000000000000000000000000B6
:10039000000000002A2B28000000000000000000E0
:1003A0000000000000000029000000002C1E342086
:1003B000212224342627252E362D3738271E1F20AC
:1003C0002122232425263333362E37381F040506F1
:1003D0000708090A0B0C0D0E0F1011121314151635
:1003E0001718191A1B1C1D2F3130232D3504050633
:1003F0000708090A0B0C0D0E0F1011121314151615
:100400001718191A1B1C1D2F3130354C0000000025
:1004100000000000000000000000000000000000DC
:1004200000000000000000000000000000000000CC
:100430007E0F00D4FFFFFFC70000007809025B00B9
:10044000030100A0FA0904000001030101000921D1
:10045000010100012244000705810308000109048D
:100460000100020300000009210101000122220015
:1004700007058403080001070504030800010904B7
:1004800002000103000000092101010001227B009C
:10049000070583030800011201100100000008C8CD
:1004A000770100010001020001140346007200619F
:1004B000006D00650077006F0072006B000000089F
:1004C000033700630038000000040309040660FFDE
:1004D0000961A1010962150026FF009520750881B8
:1004E000020963150026FF00952075089102C005DA
:1004F000010902A10185020901A1000509190129CB
:1005000008150025019508750181020501093009CA
:10051000311581257F9502750881060938158125D9
:100520007F950175088106050C0A38021581257F23
:10053000950175088106C0C005010980A1018503E8
:1005400019012AB700150126B70095017510810021
:10055000C0050C0901A101850419012AA002150199
:1005600026A002950175108100C005010906A101B0
:10057000050719E029E71500250195087501810295
:100580009501750881030507190029FF150026FF4D
:100590000095067508810005081901290515002533
:1005A00001950575019102950175039103C0112410
:1005B0001FBECFEFD8E0DEBFCDBF11E0A0E0B1E0BD
:1005C000E2E5FAE402C005900D92A03BB107D9F72D
:1005D00023E0A0EBB1E001C01D92A130B207E1F72A
:1005E0000E943C140C9427250C940000A82FB92FCE
:1005F00080E090E041E050EA609530E009C02D9144
:1006000082279795879510F084279527305EC8F349
:100610006F5FA8F30895EADF8D939D930895CF93BC
:10062000CFB7CF93DF93C3954B9BE9F74B9B10C09C
:100630004B9B0EC04B9B0CC04B9B0AC04B9B08C0F6
:100640004B9B06C0C091D802C395C093D8028EC000
:100650006F93C091D702DD27C152DD4F2F9365E51F
:100660004B9B03C02F916F91E1CF0F931F934F933B
:1006700020E040E15F9309B10C7003FB27F93F9341
:1006800050E03BE039C01C7040642F77012F5F5F62
:100690001EC0406819B11C702F7752501FC04064B3
:1006A00009B12F770C70D1F15F5F00C023C04062A9
:1006B00019B12F771C7091F15F5F00C025C00C70DD
:1006C0001027515012F45D5F0000115027952C3F08
:1006D00019B1C8F61C700127015027952C3FC8F6A8
:1006E0004227499309B10C7010274F731150279579
:1006F0002C3FA8F64695469519B11C7079F0012754
:10070000015027952C3F98F66B5A60F3315009B190
:10071000B0F600C012E01CBB00271CC03B50319556
:10072000C31BD04012E01CBB0881033C21F10B34F9
:1007300011F12091D4021981110F1213EDCF4A81CA
:10074000441F093679F10D3211F0013E29F74F703F
:1007500009F0042F0093DD023F915F914F911F91AB
:100760000F912F916F91CCB3C1FD5DCFDF91CF91F0
:10077000CFBFCF9118952091DD02222369F310910C
:10078000DB02112309F049C034300AF448C0309329
:10079000DB022093D6021091D7023BE0311B30934D
:1007A000D7023DC00091DB020130BCF50AE54F7075
:1007B00049F430911C0134FD33C000931C01C1EB9E
:1007C000D2E032C0433059F0443091F03091BC0255
:1007D00034FD26C00093BC02CDEBD2E025C03091A1
:1007E000F50234FD1DC00093F502C6EFD2E01CC037
:1007F0003091C80234FD14C00093C802C9ECD2E0A5
:1008000013C0052710E000C000000BB91AC005276F
:1008100010E0221F1DC010E021C04AE502C032EDE9
:10082000432FC4E1D0E032E01AB11C605B9A0BB1F7
:100830001AB95CE020E865E320FF05270BB927958E
:1008400017951C3FF0F66695B8F7B1F720FF05271E
:100850000BB9279517951C3FD0F62795179517FFCD
:10086000052700001C3F0BB9B0F629913A9519F7FE
:10087000037F1091DC02110FC651D0400BB911F06B
:100880001093D40212E01CBB08601AB1137F402FF2
:10089000437F54E05A95F1F70BB91AB94BB95CCFC5
:1008A000CF93DF93D82FC62F8091D3010E942006CB
:1008B000D1110AC0CC2311F041E001C040E06AE050
:1008C0000E94F4150E94020581E0DF91CF91089506
:1008D0008530B0F46B30A0F4463090F492E4899FF8
:1008E000F001112486E0689FE00DF11D1124E40F52
:1008F000F11DEE0FFF1FE850FF4F85919491089571
:1009000081E090E008959C013A9521153F4130F532
:10091000BC0166277270AC01442754709C012227E9
:10092000387094FF0FC090FF02C080E101C080E0EA
:10093000672B09F08062452B09F08064232B79F046
:1009400080680895892F8170672B09F08260452B9C
:1009500009F08460232B19F08860089580E00895E1
:10096000CF93DF93EB010E948304FE010995DF9191
:10097000CF910895CF93DF93EC01805E91090897A2
:1009800010F0209719F461E577E002C06EE779E096
:10099000CE010E94B0048C2F0E94B206DF91CF914D
:1009A0000895CF93DF93EC010E94FC06CE01805E98
:1009B0009109089710F0209719F468E577E002C0D4
:1009C00065E879E0CE010E94B004DF91CF910895EF
:1009D0000F931F93CF93DF938C01EB010E94BA0416
:1009E000209741F08FE99FE00197F1F700C00000E8
:1009F0002197F6CFC8010E94D104DF91CF911F91BA
:100A00000F9108958933910519F060E170E002C0FB
:100A100060E570E00E94E804089581E0089581E0B7
:100A200008950E940F0508950E94110508950E94DF
:100A30000F05089508950E941A050895A6E0B0E0F4
:100A4000E4E2F5E00C94832449835A839E83309139
:100A5000B70189819A81311115C03E81332359F044
:100A6000222349F00E94CB0A182F682F89819A818E
:100A70000E94A70A03C00E94B90A182F69817A81CF
:100A8000812F04C00E94CB0A69817A810E94ED11F6
:100A90002696E3E00C949F24FC01262F408151818F
:100AA00062817381848195810E941E050895CF9390
:100AB000DF93EC0161E00E944C05BE010E94140529
:100AC000DF91CF910895CF93DF93EC0160E00E9416
:100AD0004C05BE010E941B05DF91CF91089591E066
:100AE00001C0990F8A95EAF7892F0E94F0090895AD
:100AF000CF93C82F81E00C2E01C0880F0A94EAF72B
:100B00000E94330F8C2F0E946F05CF91089581E0D2
:100B100008950E9487050895CF93C82F0E94A209C7
:100B20008C2F0E9489052FEF84E39CE021508040A8
:100B30009040E1F700C00000CF91089581E00E944D
:100B40008C050E94BD20089580E00E948C050E94C3
:100B5000D22008950F931F93CF93DF938C0161E010
:100B60000E944C05EC01B8010E94C01D882309F4C5
:100B700057C0B801CE010E941705882309F450C060
:100B8000B801CE010E94971C882309F449C0B8011E
:100B9000CE010E94A217882309F442C0B801CE01F9
:100BA0000E9478178823E1F1B801CE010E94DA1C77
:100BB0008823B1F1B801CE010E94EB12882381F1A4
:100BC000F8018581882341F1C3308CE7D807D1F043
:100BD00040F4C115FCE7DF0791F0C130DC47A1F01C
:100BE0001BC0CB35ECE7DE07A9F0CC35FCE7DF070F
:100BF00071F0CA35DC4781F40E940E0F0DC00E94CF
:100C00009E050EC00E94160F0E94A40509C00E94F6
:100C1000040F02C00E94120FC8010E940D0501C0FE
:100C200080E0DF91CF911F910F9108950E94ED1FF9
:100C30000E944A0608950E944E060E94F61F0895DB
:100C4000982F92959F7019F0892F24E001C020E021
:100C5000982F9695969511F02E5F892F982F96953F
:100C600009F02F5F822F089581E008950895CF93B2
:100C7000DF93D82F0E943406C82F882319F08D2FB8
:100C80000E9436068C2FDF91CF91089508950E941F
:100C90003706089580E00E94470608950E94AE1E20
:100CA0000E9447060895CF930E94AE1EC82F8091E0
:100CB000B201C81779F0C093B2010E947C20609302
:100CC000B3017093B4018093B5019093B6018C2F5A
:100CD0000E944706CF910895ADE0B0E0E2E7F6E06C
:100CE0000C948424488759876A877B878C879D87E3
:100CF00091110E94540ECE01019627E0FC01119241
:100D00002A95E9F726E0FE013896DC0101900D9264
:100D10002A95E1F72D8121110AC029813A814B8161
:100D20005C816D817E818F810E949E0D04C00E9436
:100D300057058111F2CF2D96E2E00C94A024FC011E
:100D40002481213021F4808191810E94F80A089544
:100D5000662319F00E94121902C00E946D190E94A8
:100D6000E4190895CF93882309F444C0C82F8CEF69
:100D70008C0F813A70F48C2F0E942D1F882329F04C
:100D80008C2F0E94701F0E94A20E8C2F0E94681F41
:100D90000CC080E28C0F883058F4C77081E001C02D
:100DA000880FCA95EAF70E94370E0E94A20E22C051
:100DB000EBE5EC0FE33040F4F0E0ED5AFE4F8081BC
:100DC00090E00E94D41E16C0E8E5EC0FEB3150F421
:100DD000F0E0EE0FFF1FE35EFE4F808191810E94E5
:100DE000F91E08C083E38C0F833120F461E08C2F5F
:100DF0000E94A806CF910895882381F19CEF980F57
:100E0000913A18F40E94701F0DC090E2980F98302C
:100E100060F4877091E001C0990F8A95EAF7892FF5
:100E20000E943D0E0E94A20E08959BE5980F9330FC
:100E300028F480E090E00E94D41E089598E5980F71
:100E40009B3128F480E090E00E94F91E089593E31E
:100E5000980F933118F460E00E94A80608951F933C
:100E6000CF93DF93182FEB010E94B206209741F039
:100E70008FE99FE00197F1F700C000002197F6CFBE
:100E8000812F0E94FC06DF91CF911F910895893335
:100E900019F060E170E002C060E570E00E942F0789
:100EA0000895882321F00E94370E0E94A20E089513
:100EB000882321F00E943D0E0E94A20E0895A0E01A
:100EC000B0E0E5E6F7E00C947E247C01162FC72FF6
:100ED000FC01D581068102950F700E942D0E88239A
:100EE000F9F0DD23E9F08C2F807F803461F080E21F
:100EF000810F8830A8F08C2F807E803221F4123050
:100F000078F0002369F08091960282FF09C082E0A8
:100F10000E94D80E0E942D0E91E0D82ED92601C035
:100F2000D12CCC2EC2948FE0C8228C2D90E08C3036
:100F3000910508F088C1FC01EC5CFF4F0C9467241C
:100F40008C2F807FCF70882311F0C295C07FDD2366
:100F500099F0CC2309F45EC180E2810F883010F053
:100F6000111104C08C2F0E94370E03C08C2F0E94D9
:100F7000470E0E94A20E4EC1812F0E94FC06CC2378
:100F800009F461C180E2810F883038F1112329F121
:100F90008C2F0E944D0E24C08C2F807FCF7080320A
:100FA00011F0C295C07F112319F0113099F13CC0A6
:100FB0008091960282FD17C0DD2349F0CC2329F0F1
:100FC0008C2F0E94370E0E94A20E80E024C180E088
:100FD0000E94FC06CC2309F436C18C2F0E943D0EE2
:100FE0000E94A20E30C1DD2349F0002309F1013037
:100FF00009F029C18C2F0E945E0E25C1011123C169
:101000008C2F0E9458078C2F0E946A0E8C2F0E94F2
:10101000AB0E19C1DD2321F0063008F014C108C061
:10102000053008F010C10AC0DD2331F00111F2C013
:101030008C2F0E94510707C10111F2C08C2F0E9412
:10104000580701C18C2F86958695837019F08130E1
:1010500061F0F9C0DD2321F0812F9C2F937002C035
:1010600080E090E00E94D41EF6C0DD2321F0812FA5
:101070009C2F937002C080E090E00E94F91EEBC0AC
:101080006D2F812F0E94A806E6C08C2F837079F502
:10109000D111DDC0412F429546954770440F440F52
:1010A000212F2F70042E01C0220F0A94EAF714FF9B
:1010B00008C08FE090E001C0880F4A95EAF780955C
:1010C00001C080E0C695C695C370822BC23049F03E
:1010D00058F4C13019F00E94F909B9C00E94F3090F
:1010E000B6C00E94FF09B3C00E94F009B0C0DD2362
:1010F00019F08C2F817001C08695882309F4A7C050
:10110000412F429546954770440F440F212F2F7071
:10111000042E01C0220F0A94EAF714FF08C08FE0E2
:1011200090E001C0880F4A95EAF7809501C080E001
:10113000C695C695C370822BC23049F058F4C130B1
:1011400019F00E94450A83C00E943F0A80C00E9495
:101150004B0A7DC00E94080A7AC0CF70DD2339F0A7
:101160008C2F0E941A0A812F0E94510770C0812F74
:101170000E9458078C2F0E94260A69C0123F21F155
:1011800028F4103F41F0113FC1F040C0133F19F166
:10119000143F79F03BC0DD2341F0053008F053C027
:1011A0008C2F8F710E94330A4EC0063008F04BC05E
:1011B000F7CF8091960282FD18C0DD2339F08C2F85
:1011C0008F710E941A0A3FC0DD23C9F38C2F8F71E3
:1011D0000E94260A38C0DD2329F08C2F8F710E94CF
:1011E000110A31C00E940D0A2EC0DD2331F063E0E8
:1011F0008C2F8F710E94BA0E26C081E00E94D80EFB
:10120000023008F182E00E94D80E1DC0DD2331F0CB
:101210000023A9F2812F0E94B20615C00023B1F26B
:10122000193341F4FFEF27EE83E0F1502040804076
:10123000E1F704C0EFEFF9EF3197F1F700C00000DC
:10124000812F0E94FC0688EF8C0D843020F40E94D0
:10125000AE1E0E944706DD2089F00E94290E80FD07
:101260000DC0F70115820E94230E0E941A0AC701C1
:101270000E945B090E94230E0E94260ACDB7DEB7AA
:10128000E8E00C949A240F931F93CF93DF93EC0123
:10129000688179818D810E94030B8C010E94510A23
:1012A0000E94E309B801CE010E945F07DF91CF9150
:1012B0001F910F910895CF93DF93FC012481222386
:1012C000D1F0EC010E94AA0581110FC00E942D0EE1
:1012D000882389F08D81882371F08091960282FFA6
:1012E0000AC082E00E94D80E06C0CE010E944309C7
:1012F000CE010E946305DF91CF910895882321F0EC
:101300000E94470E0E94A20E0895882321F00E9499
:101310004D0E0E94A20E089580E090E00E94D41E1F
:1013200080E090E00E94F91E0E94540E0E94A20EDE
:101330000E94031A0E94E41908950E94781F0E94D7
:101340008C0908950E94440E0E949D09089592956B
:101350009F70963079F010F4925001C09A509230FC
:1013600068F4803F69F018F4883E40F409C0843F77
:1013700029F406C0883E20F0813F11F080E00895F6
:1013800081E00895FC012481222339F0808191813C
:101390000E94F80A0E94A709089580E00895A6E037
:1013A000B0E0E5EDF9E00C9484242696E2E00C949C
:1013B000A024A7E0B0E0EFEDF9E00C948424279698
:1013C000E2E00C94A024089508950E94E409089591
:1013D0000E94E50908950E94E8098093D4010895C8
:1013E0000E94EB0908959091D401892B0E94EB098A
:1013F00008959091D40189230E94EB09089590915A
:10140000D40189270E94EB0908950E94E4090895F8
:101410000E94050A8093D301089580E00E94080A83
:10142000089591E001C0990F8A95EAF7892F0E94EB
:10143000080A089521E030E001C0220F8A95EAF7FA
:101440008091D301822B0E94080A089521E030E0A8
:1014500001C0220F8A95EAF720958091D30182235B
:101460000E94080A089521E030E001C0220F8A9509
:10147000EAF78091D30182270E94080A089590918B
:10148000D301892B0E94080A08959091D3018923E2
:101490000E94080A08959091D30189270E94080AA2
:1014A00008950895962F9770A1E001C0AA0F9A950C
:1014B000EAF793E0769567959A95E1F7FB01EE0FD1
:1014C000FF1F6E0F7F1FFA01E60FF71F40E050E08D
:1014D000682F70E090819B01042E02C036952795FD
:1014E0000A94E2F72170219529272A23292721939D
:1014F0004F5F5F4F4330510569F708959B01782F87
:10150000777043E0969587954A95E1F7FC01EE0FD9
:10151000FF1F8E0F9F1FF901E80FF91F40E050E0F9
:1015200080E0219130E0072E02C0369527950A947D
:10153000E2F721703327042E01C0220F0A94EAF744
:10154000822B4F5F5F4F4330510559F70895282F85
:101550009B3070F4863060F4862F622F70E026E0B6
:10156000929F600D711D112448EB51E00E94520AB8
:1015700008959B3070F4863060F4292F90E068EB7A
:1015800071E036E0239F800D911D11240E947E0A98
:10159000089580E00895CF92DF92FF920F931F93FA
:1015A000CF93DF936C010091D3018091D401082B7C
:1015B000C4E0D0E010E0C8010C2E02C095958795DC
:1015C0000A94E2F780FD04C02197A8F7F12C07C028
:1015D000FC2EB6018C2F0E94F9110197A9F38F2DD3
:1015E000DF91CF911F910F91FF90DF90CF900895E1
:1015F000CF93DF93EC010E94CB0ABE010E94F91148
:10160000DF91CF9108951F93CF93DF93EB019091DA
:10161000B701992321F0CB010E94F80A13C0882357
:1016200049F0CB010E94CB0A182F682FCE010E94EF
:10163000A70A04C0CB010E94B90A182FBE01812F4E
:101640000E94F911DF91CF911F910895E1E0F0E040
:10165000DF0102C0AA0FBB1F6A95E2F7BD01DF01DF
:1016600002C0AA0FBB1F4A95E2F7AD01462B01C08D
:10167000EE0F2A95EAF7942F9823491302C08E2B78
:101680000895E0958E230895242F462F682F80918A
:10169000D3010E94260B0E94080A08951F93CF933E
:1016A000DF93C091D50117E08091D601C817A1F052
:1016B000D0E01C9FF0011D9FF00D1124E952FE4F58
:1016C00020813181428153816481758186810E94AC
:1016D000D9092196C770E8CFDF91CF911F91089566
:1016E00020910F023091100240911102509112028C
:1016F0006091130270911402809115020E94D90921
:101700000895CF93DF938091150282958F7009F031
:101710004EC080911402882309F449C08091D501FC
:101720004091D6015091100260910F02C0911102B8
:10173000D091120277E08417D1F190E0789FF00108
:10174000799FF00D1124DF01A952BE4F14962C9100
:101750001497222349F111962C911197251324C037
:101760002C91261321C015962C91159721111CC080
:1017700012962D913C9113972C1B3D0B283C310563
:1017800098F4809115028F70806180931502E35266
:10179000FE4F80818F70806180838FE092E00E9495
:1017A0005B090E944E0B03C001968770C4CFDF9186
:1017B000CF9108952091D5019091D60157E0291736
:1017C000A9F030E0529FF001539FF00D1124E9522F
:1017D000FE4F7181761306C07081781303C0758146
:1017E000741306C02F5F3F4F2770E9CF80E0089544
:1017F00081E00895A4E1B0E0E0E0FCE00C947A24FC
:101800008C0186E0F801DE011F9601900D928A9509
:10181000E1F7F8018481E5809FE0A92E92E0B92EDE
:1018200090911302911118C0882309F480C1EE2011
:10183000D9F1C8010E94C209F82E8823A9F187E0D6
:10184000F801D50101900D928A95E1F7C5010E943A
:101850009F060E94810B98C0F801C080D1808280D1
:101860009380F09014022091110230911202A40191
:10187000421B530BFF2009F406C1483C510508F0F8
:10188000AFC0882309F455C180911502282F207F0D
:1018900090911002222361F09D1509F462C0C801E5
:1018A0000E94C209811173C0C8010E945B093FC137
:1018B0009D1115C090910F029C1111C0E1100FC035
:1018C0008F708061809315020E94700B8FE092E010
:1018D0000E945B0980911502F801868326C1E11000
:1018E0003AC040E06D2D8C2D0E94DA0B40E06D2D4A
:1018F0008C2D0E94DA0BE82E811117C1CF86D88A71
:101900008F8598890E94F80A292F22952F702430FC
:1019100020F49F70223028F009C02A50223080F035
:1019200014C0992349F0811107C013C0992321F0F5
:10193000F8019681907F69F0805E883030F409C0AC
:10194000803F38F0815F833020F0C8010E945B093E
:10195000EF2CFE2CEEC08091150281608093150261
:10196000E4C090910F029C119ACFE11098CFF8013A
:101970008683C8010E945B0987E0F801AFE0B2E00E
:1019800001900D928A95E1F70E94700BD2C0EE2073
:1019900009F48ACF20911502822F82958F7090E0F2
:1019A00002978CF080910F0290911002998788879E
:1019B0009B868A86809113028C871D862E87CE0196
:1019C00008960E945B0987E0F801AFE0B2E0019061
:1019D0000D928A95E1F70E94810B0E94700BA7C0BF
:1019E00090911502292F207FA1F4682D9A8A898A67
:1019F000A6017A899E2D0E94CF098FE092E00E9475
:101A00005B0987E0F50111928A95E9F70E94700B56
:101A10008CC0882309F48DC0809110028D1111C0F3
:101A200080910F028C110DC0E1100BC0F80196835C
:101A3000C8010E945B0987E0F50111928A95E9F7D8
:101A400078C0C8010E94C209882309F42DCFEE2076
:101A500009F42ACF20911502822F82958F7090E091
:101A600002970CF4B0CF80910F02909110029A83EC
:101A700089839C828B82809113028D831E822F83A7
:101A8000CE0101969ECF483C510508F040C0882306
:101A900009F44DC0FE2CEE2009F406CF809110020F
:101AA0008D1127C080910F028C1123C090911502D7
:101AB00090FD16C0892F82958F70282F30E0211558
:101AC000310571F0F80196832F30310509F451CFBB
:101AD0008F5F982F9295907F86818F70892B48CF4A
:101AE00087E0F801AFE0B2E001900D928A95E1F74E
:101AF00020C0C8010E94C209811165CF80911502E2
:101B0000816080931502C8010E945B0912C0682D94
:101B10009A8A898AA6017A899E2D0E94CF0987E038
:101B2000F50111928A95E9F72FCFF12C02C0FF241D
:101B3000F3948F2D6496ECE00C949624AEE0B0E024
:101B4000E4EAFDE00C948324288739874A875B8781
:101B50006C877D878E87CE0108960E94FA0B8823BA
:101B600061F06C856623A9F1288539854A855B85F6
:101B70007D858E850E94D9092CC087E0FE013896AC
:101B8000DE01119601900D928A95E1F76C8566232E
:101B900001F12091D60130E0C901019687709927A3
:101BA0004091D50150E084179507E1F16D8397E0EE
:101BB000929FD001939FB00D1124A952BE4FFE01F8
:101BC000319601900D929A95E1F78093D6010E948B
:101BD0004E0B17E08091D5019091D601891779F1CC
:101BE000189FC001112489529E4F0E94FA0B88232E
:101BF00031F1E091D5011E9FF0011124E952FE4F11
:101C000020813181428153816481758186810E9466
:101C1000D9098091D50190E001968770992780932A
:101C2000D501D8CF0E94A2091092D6011092D501F9
:101C3000EFE0F2E087E0DF011D928A95E9F72E964A
:101C4000E3E00C949F2480911602869586958695F4
:101C500008958091160287700895909116029770EA
:101C600081E009F480E00895809122020895909126
:101C70002202892B8093220208958095909122025E
:101C80008923809322020895109222020895909150
:101C90002102892B80932102089580959091210241
:101CA00089238093210208951092210208950895B6
:101CB0000E94570E08950E94580E089590911802A0
:101CC000292F2823821729F0982B909318020E941D
:101CD0005B0E089590911802292F282331F08095EA
:101CE0008923809318020E945B0E08958091180248
:101CF000882329F01092180280E00E945B0E08955C
:101D00000F931F93CF930091000110910101C09197
:101D1000220280912102C82B80911802882331F081
:101D2000C82B0E941E1F81110E94760EF801C083ED
:101D300080910001909101010E94BB1ECF911F91E3
:101D40000F9108950E94800E08950E94570E0895E5
:101D50000E94A50E089590911702292F282331F093
:101D600080958923809317020E94A80E08950E94EF
:101D7000570E08959091960292FF11C098E0899FA6
:101D800090011124262B209316020E941A0A80919A
:101D900016028695869586950E94B70E08950E9434
:101DA0001A0A08951092160280E00E94B70E089554
:101DB000909116028095892380931602282F277010
:101DC00069F4981759F09091960292FF07C0869592
:101DD000869586950E94260A0E94D20E08959091BB
:101DE000960292FB222720F9281769F080FB92F9CE
:101DF0009093960280919502909196020E943E0FD8
:101E000082E00E94D80E08958091960282FB882776
:101E100080F991E089270E94EF0E089581E00E94E9
:101E2000EF0E089580E00E94EF0E08956FEF7FEFB0
:101E300080E090E00E941125089580E090E00E94EB
:101E4000DD24853E9E4F19F40E94251D089580E0F3
:101E5000089582E090E00E94D524089583E090E008
:101E60000E94D5240895682F83E090E00E94F32417
:101E7000089584E090E00E94DD240895BC0184E090
:101E800090E00E9411250895AB01BC018FE090E025
:101E90000E9405250895AB01BC0183E190E00E94FA
:101EA0000525089560E070E0CB010E944B0F089576
:101EB00060E070E0CB010E94440F0E94520F089531
:101EC000A8E0B0E0E6E6FFE00C94842465EE7EEF47
:101ED00080E090E00E94112560E082E090E00E94A6
:101EE000F32481E08093D4010E94330F60E074E119
:101EF00084E090E00E94112560E086E090E00E947E
:101F0000F32460E087E090E00E94F32440E050E09A
:101F1000BA0188E090E00E94052560E083E290E04D
:101F20000E94F32460E08CE090E00E94F32460E0E3
:101F30008DE090E00E94F32419821A821B821C8299
:101F40001D821E821F82188648E050E067E170E023
:101F5000CE0101960E94E32440E050E0BA018FE1F7
:101F600090E00E94052580E00E943E1D0E94A21D77
:101F70000E94580F2896E2E00C94A0240E94600F63
:101F80000895682F8EE090E00E94F3240895A6E063
:101F9000B0E0EDECFFE00C9482240E9470208C01F4
:101FA00080912302909124020817190781F0198269
:101FB0001A820E947020682F49815A81792F80E00F
:101FC00090E00E946C061093240200932302269650
:101FD000E4E00C949E240E947C206093380270936D
:101FE000390280933A0290933B02609334027093DB
:101FF0003502809336029093370208950E947C2028
:10200000609338027093390280933A0290933B02B6
:1020100060933002709331028093320290933302C6
:10202000089581E0089581E008950E9413100895B5
:1020300008950E94181008950E94181008950E9493
:102040001C1008950E94181008950E9422100895EF
:102050000E941810089589EE92E10E9453140E9484
:1020600028100E94251008950E9419100E9418102F
:1020700008950E941D0F811102C00E94BE0F0E9490
:10208000290F80933C020E94390F9093960280930F
:1020900095020E94DE150E942E0F0E94F009809189
:1020A000D3010E94050A08950E9467200E94B21D74
:1020B0000E945B140E94B0130E9439100E944606D1
:1020C0000E941F100895A6E0B0E0E9E6F0E10C944C
:1020D0007B240E941110811103C00E94C70F53C0BE
:1020E0000E94C61385E2E82E82E0F82E670100E028
:1020F000F60111916F01802F0E94FE1281270F5F60
:102100000B3019F08823A1F302C0882331F38091AA
:102110003C0281FD0E9404130E941510A82E10E0BD
:1021200099249394812F0E94FE12B82EF701C0804B
:10213000C82609F100E0DD24D3948C2D8D21A9F06F
:10214000AA2099F009831A830E9470209C838B83B4
:102150009D8291E08B2D8D2109F490E049815A8177
:102160006B817C818D810E946C060F5FDD0C0630D7
:1021700021F7F701B0821F5FFFEFEF1AFF0A1B3054
:1021800089F60E94EB0F0E94D81481110E94FE0F65
:102190000E94251A0E9453062696EBE00C94972481
:1021A0001F93CF93DF930E94FE11EC01C11580E5D0
:1021B000D807E8F5C11590E4D90708F0A8C0C03EDB
:1021C000D10530F5CD3CD10508F094C0C83AD10511
:1021D00078F4C53AD10508F083C0C130D10509F4BF
:1021E0007CC008F4F2C0C430D10508F0F1C0EDC0E5
:1021F000C33CD10508F0E9C0C85AD0E0CC0FDD1FC0
:10220000CA5ADE4F0990D881C02DCE019464E1C036
:10221000C11580E2D80708F0CBC0C11591E0D907FD
:1022200008F06BC0C83ED10508F4D2C0CEC0C0369D
:1022300082E5D80728F5C03492E5D90708F079C0BF
:10224000C03282E5D80708F06CC0C11592E5D90705
:1022500008F481C04C2F4695469580E2489FA00126
:102260001124C37021E030E0C90102C0880F991F1A
:10227000CA95E2F7EA01C82BD92BCE019D68A9C007
:10228000C03A82E5D807B8F48C2F8F71C03892E538
:10229000D90708F07BC08695869590E2899F9001CA
:1022A0001124C37081E090E002C0880F991FCA9585
:1022B000E2F79A6868C0C03C82E5D80708F46DC0B0
:1022C000C03E92E5D90708F080C0CF71DD27DC2F32
:1022D000CC27CE01806F906A7CC081E090E079C00D
:1022E000C55AD0E0C457DE4F8881C82FD0E0CE0158
:1022F00090646FC0CE0190656CC08D2F0E949A12C1
:10230000182FCE0199270E94FE111F715CC0CE01CB
:1023100099270E94FE11CC27DF70D06A8C2B9D2B51
:1023200058C0CF71D0E0DC2FCC27CE01816F906AEE
:1023300050C08C2F8F718695869590E2899F900171
:102340001124C37081E090E002C0880F991FCA95E4
:10235000E2F79C6818C08C2F8F710E949A1295E04A
:10236000D695C7959A95E1F7CF70D0E0DC2FCC27B2
:10237000282F30E084FF05C084E0220F331F8A95A8
:10238000E1F7D069CE01822B932B23C090E0D82FA8
:10239000CC27CE01846F906A1CC08C2F8F710E9455
:1023A0009A128F7190E0D82FCC27CE01906211C085
:1023B0008D2F8F710E949A12182FCE0199270E949B
:1023C000FE111F719062912B04C080E090E001C06B
:1023D000CE01DF91CF911F9108957B3038F46630A4
:1023E00028F4462F672F0E949016089580E090E011
:1023F00008950E94ED110E94D01008958238910531
:1024000069F1B0F48133910509F475C048F489325B
:10241000910509F467C08A32910509F471C00895E5
:102420008533910509F459C089339105B9F00895B0
:10243000833E910589F138F4803E9105D1F0823ECA
:10244000910529F10895863E9105C9F1873E9105D0
:10245000D9F1843E910509F06CC027C02091950206
:1024600020FD57C021FD55C02091960223FD5BC081
:1024700008958091950280FD48C08091960280FF6A
:1024800048C08091950284FD46C083EE51C0809182
:10249000950282FF3CC0F5CF8091950282FD37C046
:1024A0008091960280FD35C0ECCF8091960281FF2D
:1024B00036C08091950284FD2EC087EE39C0809190
:1024C000950283FF2AC0F5CF8091950283FD25C038
:1024D0008091960281FD23C0ECCF8091950285FD0D
:1024E00022C01FC08091950285FD1BC0809196027D
:1024F00083FF19C00AC08091950286FD16C017C0DF
:102500008091950286FD13C010C089E311C082EE50
:102510000FC080EE0DC080E00BC086EE09C084EED7
:1025200007C085E305C089E203C08AE201C081E3F8
:1025300090E008959091950292FF10C041E0282FFD
:102540002471243009F040E031E0282F2871283030
:1025500009F030E0431711F02CE0822793FF10C000
:1025600041E0282F2471243109F040E031E0282F88
:102570002871283109F030E0431711F02CE0822750
:102580003091960230FF10C051E0282F2171213088
:1025900009F050E041E0282F2871283009F040E090
:1025A000541711F029E0822731FF10C041E0282F95
:1025B0002171213109F040E031E0282F28712831C4
:1025C00009F030E0431711F029E0822794FD877E5F
:1025D000089580E00895CF939C01205E324520321B
:1025E000310540F4FB01C581C11105C08F710E9406
:1025F000780501C0C1E08C2FCF910895E82FF0E05D
:10260000EE55FD4F80810895089580EA8A95F1F78F
:10261000089500C008950E940513089508950E942A
:102620000E1308950E940F1308950E940E1308952B
:102630000E9415130895F894E82FE295EF70F0E0EA
:1026400031A1282F2F7081E090E001C0880F2A95DA
:10265000EAF7982F9095932391A392A1892B82A3B7
:10266000789408950F931F93CF93DF93C5E9D1E03A
:1026700089918F3F11F00E941B1381E0C03AD80767
:10268000B9F7CFE8D1E005E911E089918F3F11F06A
:102690000E941B130C171D07C1F7DF91CF911F91EB
:1026A0000F910895A0E0B0E0E8E5F3E10C947E24FA
:1026B0008C01C62FD0E0CE018B569E4F7C01FC01D1
:1026C00090819F3F09F447C0D62EF894E92FE295F8
:1026D000EF70F0E081A19F7021E030E001C0220F97
:1026E0009A95EAF7822B81A382A12095282322A321
:1026F00078940E940913EFE8F1E045E951E031E0F8
:10270000C12C21912F3F89F0A22FA295AF70B0E08C
:1027100090968C9190E02F7002C0959587952A95A0
:10272000E2F780FD02C0832F01C080E0C82A330F8A
:102730004E175F0731F7F70180818F3F11F00E943C
:102740001B1361E0C11001C060E08D2D0E940B13CE
:10275000C00FD11FC882CDB7DEB7E8E00C949A2431
:102760000E9432138BE0E2EAF2E0DF01982F1D9223
:102770009A95E9F7E7E9F2E0DF011D928A95E9F71A
:102780008BE00E9401140E9418130895ABE0B0E0A2
:10279000ECECF3E10C9481248E010F5F1F4F8BE072
:1027A000F80111928A95E9F7F12C6F2DC8010E946A
:1027B0005213F394FBE0FF12F8CF4BE050E0B80166
:1027C00087E992E00E94BF2421E0009709F420E00D
:1027D000892B41F08BE0F801A7E9B2E001900D925E
:1027E0008A95E1F74BE062EA72E087E992E00E94A5
:1027F0000214182F0E941213812F2B96E5E00C94DF
:102800009D240895EF92FF920F931F93CF93DF9330
:102810007C018B01C42F222351F081E080933F0281
:102820000E94702090933E0280933D0204C08091EC
:102830003F02811102C080E01AC080913D02909158
:102840003E020E9488200597B0F3D0E0AE01B701A8
:10285000C8010E94BF24892B39F0AE01B701C8011D
:102860000E94CC2481E001C080E010923F02CDB7ED
:10287000DEB7E6E00C949C240E940D200E94FE200E
:102880000E942B100E940E210E9454100E941F21B2
:102890000E942D210E945A210E9466210E94FA2145
:1028A0000E943410F5CF9093B1018093B001089548
:1028B0000E941310089588E0E1E4F2E0DF011D9228
:1028C0008A95E9F70E9463150895FC01228130E0A2
:1028D0002F5F3F4F23703327438150E081E024175F
:1028E000350709F080E008950F931F93CF93DF938E
:1028F000EC01162F042F0E946514811113C08A81E8
:10290000FE01E80FF11D1F7764816078612B00FBE9
:1029100067F964838F5F83708A8388818F5F888380
:1029200081E001C080E0DF91CF911F910F91089568
:10293000FC01838192819817B1F0DF01A80FB11DCE
:1029400014968C9187FB992790F98F77DB018C93F4
:10295000DA019C9383818F5F8370838381818F5F92
:10296000818381E0089580E00895462F682F81E4F7
:1029700092E00E9474140895AB01BC0181E492E0DE
:102980000E9498140895CF93DF93D62F0E9450048D
:10299000C82F882349F06AE070E0DD2311F089EA4E
:1029A00001C08AEA0E942F078C2FDF91CF910895F2
:1029B000A2E0B0E0EEEDF4E10C94832480914002BB
:1029C000882351F010924002809143028093440288
:1029D00080914102809342020E94A6150E945814E1
:1029E00010E0882379F0BE016F5F7F4FCE01029621
:1029F0000E94BC14882331F069818A810E94C3142B
:102A000011E0F1CF812F2296E3E00C949F248FE810
:102A100091E00197F1F700C000000895611102C034
:102A200080E901C081E93AB1282F2F7081E090E060
:102A300001C0880F2A95EAF7982F909593239AB9A9
:102A40009BB1892B8BB90895611102C020E901C0A7
:102A500021E989B190E02F7002C0959587952A955C
:102A6000E2F7817008950895CF93DF93C0E08091DD
:102A70004902C81750F460E08C2F0E940E1561E0E7
:102A80008C2F0E940E15CF5FF2CF0E940715C0E079
:102A900080914902C81790F460E08C2F0E942415A1
:102AA000D82F61E08C2F0E942415EC2FF0E0E55B1D
:102AB000FD4F880FD82BD083CF5FEACF0E9433150C
:102AC000DF91CF91089581E0809349020E943415EF
:102AD00008951F93CF93DF93E42FEE0F6E2BC82F33
:102AE000D0E0DE01A55BBD4FEC912E2F237030E0CE
:102AF000462F50E02417350729F1182FEE0FEE0F5F
:102B0000E62BEC93EF70F0E0E056FE4FC65BDD4F36
:102B100090818881890F8883843024F060E0812F40
:102B20000E94B51488818D3F24F461E0812F0E94BA
:102B3000B5148881082E000C990B64E070E00E94A7
:102B400053248883DF91CF911F910895CF93DF9312
:102B5000C0E080914902C81780F461E08C2F0E9488
:102B60002415D82F60E08C2F0E9424154D2F682F3C
:102B70008C2F0E946915CF5FECCFDF91CF91089524
:102B80000E94160F089580E00E94FE128170089541
:102B90000E94C6132FEF86E791E0215080409040BD
:102BA000E1F700C000000E94C6130E94C3158823ED
:102BB00021F00E94C0150E94BD2008950E94C815F2
:102BC000089585E0089550E0440F551F2CE0629F62
:102BD000400D511D11249A0164E8869F200D311D7E
:102BE0001124C9018A9608950F931F93CF93DF9301
:102BF0008530A0F46B3090F4463080F40E94E315E9
:102C00008C010E94D52490E0D82FCC27C8010196D2
:102C10000E94D5249E01282BC90102C080E090E0CB
:102C2000DF91CF911F910F9108950F931F93CF9331
:102C3000DF93853080F46B3070F4463060F4E90146
:102C40000E94E3158C016D2F0E94F3246C2FC801A4
:102C500001960E94F324DF91CF911F910F91089567
:102C60001F93CF93DF93D0E0C0E010E0412F6C2F93
:102C70008D2F0E9468049C01412F6C2F8D2F0E9484
:102C800015161F5F163091F7CF5FCB3071F7DF5FFE
:102C9000D53051F7DF91CF911F910895EF92FF92B8
:102CA0000F931F93CF93DF93EA017A01E60EF71E8D
:102CB0008C01C8018A96CE15DF0569F0043922E03F
:102CC000120720F40E94D524888301C0188221961F
:102CD0000F5F1F4FEECFCDB7DEB7E6E00C949C241C
:102CE000EF92FF920F931F93CF93DF93EA017A0144
:102CF000E60EF71E8C01C8018A96CE15DF0559F045
:102D0000043922E0120718F468810E94F324219606
:102D10000F5F1F4FF0CFCDB7DEB7E6E00C949C24D9
:102D2000853038F46B3028F4463018F40E94F415DE
:102D3000089580E090E0089580E1089582E491E0B4
:102D40000895EF92FF920F931F93CF93DF93EA01C1
:102D50007A01E60EF71E8C01C80182549D4FCE15F4
:102D6000DF0569F0023421E0120720F40E94D52427
:102D7000888301C0188221960F5F1F4FEDCFCDB71A
:102D8000DEB7E6E00C949C24EF92FF920F931F9322
:102D9000CF93DF93EA017A01E60EF71E8C01C8019A
:102DA00082549D4FCE15DF0559F0023421E0120701
:102DB00018F468810E94F32421960F5F1F4FEFCF14
:102DC000CDB7DEB7E6E00C949C24CF93DF93CEEB37
:102DD000D2E060E0CE010E94F3242196C11584E088
:102DE000D807B9F7DF91CF910895A8E0B0E0EBEFF5
:102DF000F6E10C947A24F82E8FE08F1508F474C055
:102E00008FEF93E00E94D52481116EC00EEB12E08B
:102E1000FF2071F0011594E0190709F465C0C8019D
:102E20000E94D524811101C0FA940F5F1F4FF0CF8B
:102E3000FE0131966F0188E011928A95E9F77801D9
:102E4000FFEFEF1AFF0AC8010E94D52489831A8276
:102E5000882309F449C0813009F040C0580182E05C
:102E6000A80EB11CC7010E94D5248A838823E1F1F2
:102E70009FEF980F933060F4780193E0E90EF11C16
:102E8000C5010E94D5248B83882371F11C8226C042
:102E9000843019F54E01E3E08E0E911C02E010E043
:102EA0007501FFEFEF1AFF0AC5010E94D524F40156
:102EB00081934F018823C1F08C3741F4E2E0F0E0C8
:102EC000EC0FFD1FE00FF11F108208C00F5F1F4FB6
:102ED00057010730110521F707C0750160E1C601F0
:102EE0000E94C51B8701ABCF2896ECE00C9496247A
:102EF000CF93DF9386319C4709F5EB010E94340E96
:102F00009D81992371F08A7A91E009F490E0909381
:102F10004C02811102C089E201C085E30E94681F52
:102F200009C080914C02811102C089E201C085E391
:102F30000E94701F0E94A20E80E001C081E0DF911C
:102F4000CF910895CF93DF93FC01DB0115968C910F
:102F5000882309F4DDC09F0130572332310508F082
:102F6000D8C0EF010E94390F90939602809395028A
:102F7000FE01E150F047E232F10520F4E05CFF4F42
:102F80000C946724809195028160AAC0809196027A
:102F90008860B2C0809195028260A2C08091950243
:102FA00020C08091950288609BC0809196021EC0CF
:102FB000809196028260A0C080919502806190C04D
:102FC0008091950280628CC080919502806488C057
:102FD0000E94A20980919502806882C0809195022A
:102FE000886084607DC0809196028260816084C028
:102FF000809195028E7F74C080919602877F7CC0FD
:10300000809195028D7F6CC08091950220C0809147
:103010009502877F65C0809196021EC080919602BE
:103020008D7F6AC0809195028F7E5AC080919502F3
:103030008F7D56C0809195028F7B52C00E94A2095D
:10304000809195028F774CC080919502877F8B7F0E
:1030500047C0809196028D7F8E7F4EC080919502F1
:1030600082FB222720F991E0922790FB82F990FBC6
:1030700083F936C080919602982F909591708E7F3B
:10308000892B90FB81F938C08091950286FB22271D
:1030900020F991E0922790FB86F922C00E94A209B4
:1030A0008091950287FB222720F991E0922790FBDF
:1030B00087F916C081E001C080E00E94C10F1EC0E8
:1030C0008091950284FB222720F991E0922790FBC2
:1030D00084F906C080919502982F909590FB80F915
:1030E000809395020BC08091960283FB222720F9E2
:1030F00091E0922790FB83F980939602809195024C
:10310000909196020E943E0F0E94A20980E001C0A9
:1031100081E0DF91CF910895282F35EB2303C00183
:10312000112497FF03C08058910902C080589F4F17
:10313000892F08958091530280FF06C06091070196
:1031400070E0660F771F26C081FF04C06091070101
:1031500084E005C082FF07C06091070188E0689F96
:10316000B001112417C0909152029923D1F06091BF
:103170000601961788F72091070188E0289F9001A3
:103180001124929FA001939F500D112470E0CA0159
:103190000E9453246038710540F46115710519F4DB
:1031A00006C068E070E0862F08958FE7089581E0FB
:1031B00008958091530280FF08C06091030170E080
:1031C000759567957595679521C081FF06C06091DB
:1031D000030170E07595679519C082FF04C0609186
:1031E000030170E010C090915102992399F0609111
:1031F00002019617A0F780910301899FC001112455
:1032000070E00E9453246038710540F46115710527
:1032100019F406C061E070E0862F08958FE70895E5
:1032200081E008958D3C21F40E949A18819504C094
:103230008E3C29F40E949A188093570208958F3C7F
:1032400021F40E949A18819504C0803D29F40E94BF
:103250009A18809356020895893D19F40E94D9184E
:1032600005C08A3D31F40E94D91881958093580297
:1032700008958B3D21F40E94D918819504C08C3D9E
:1032800029F40E94D9188093590208959FE2980F5B
:10329000983078F421E030E0A90102C0440F551FB6
:1032A0009A95E2F7CA0190915502892B80935502B5
:1032B00008958D3D21F48091530281600BC08E3DB5
:1032C00021F480915302826005C08F3D29F48091E2
:1032D000530284608093530208958D3C39F4909199
:1032E000570297FF35C01092570259C08E3C29F4FF
:1032F000909157021916BCF32BC0909156028F3C47
:1033000029F497FF25C01092560249C0803D19F458
:103310001916CCF31DC090915802893D29F4191655
:10332000BCF4109258023BC08A3D19F497FF10C0BC
:10333000F8CF8B3D39F49091590297FF09C0109254
:1033400059022DC08C3D21F4909159021916BCF3FD
:103350009FE2980F983080F421E030E0A90102C08C
:10336000440F551F9A95E2F7CA0180959091550236
:1033700089238093550213C08D3D21F4809153021F
:103380008E7F0BC08E3D21F4809153028D7F05C04E
:103390008F3D29F4809153028B7F8093530280915B
:1033A0005602811106C080915702811102C010920D
:1033B000520280915802811106C0809159028111F8
:1033C00002C01092510208950E947020209156026E
:1033D000211104C020915702222321F09093500222
:1033E00080934F0220915802211104C0209159026C
:1033F000222321F090934E0280934D0284E592E0C7
:103400000E94C61E0895E4E5F2E086E0DF011D9209
:103410008A95E9F7109252021092510210925302CB
:103420000895FC01828181110DC0838181110AC040
:103430008481811107C091E08581811101C090E0F4
:10344000892F01C081E081700895A6E0B0E0EBE231
:10345000FAE10C94832486E0E4E5F2E0DE011196C3
:1034600001900D928A95E1F7109256021092570240
:1034700010925802109259028B81811104C08C81E4
:10348000882309F456C080914F02909150020E9407
:103490008820AC0190915202992339F020910801C3
:1034A00030E02417350758F044C0209109018AE024
:1034B000289F900111242417350718F03AC09F3F28
:1034C00019F09F5F909352021B81112361F00E94BB
:1034D0009A18111614F09FEF01C091E0989F902D5B
:1034E0001124909356021C81112361F00E949A18B6
:1034F000111614F09FEF01C091E0989F902D1124B8
:103500009093570280915602882399F010915702A8
:10351000112379F00E948C18811101C081E0809301
:103520005602812F0E948C18811101C081E0809386
:1035300057028D81811104C08E81882309F456C001
:1035400080914D0290914E020E948820AC01909192
:103550005102992339F02091040130E024173507F6
:1035600058F044C0209105018AE0289F9001112461
:103570002417350718F03AC09F3F19F09F5F9093CA
:1035800051021D81112361F00E94D918111614F007
:103590009FEF01C091E0989F902D112490935802C5
:1035A0001E81112361F00E94D918111614F09FEFAB
:1035B00001C091E0989F902D112490935902809121
:1035C0005802882399F010915902112379F00E9432
:1035D0008C18811101C081E080935802812F0E94D4
:1035E0008C18811101C081E080935902BE016F5F88
:1035F0007F4F84E592E00E94831F811105C084E51E
:1036000092E00E94111A81110E94E41986E0FE01E5
:103610003196A4E5B2E001900D928A95E1F72696E5
:10362000E3E00C949F248F929F92BF92CF92DF92FF
:10363000EF92FF920F931F93CF93DF93E82FF0E069
:10364000E457FC4FB490282F26952695269530E018
:10365000F901E45DFB4FE4908770F12C082E02C065
:10366000F594E7940A94E2F791E0E922FF24F90146
:10367000E45EFB4FC490D12C082E02C0D594C794B1
:103680000A94E2F7E1E0CE22DD24F901E45FFB4F8A
:10369000C491D0E002C0D595C7958A95E2F7C17074
:1036A000DD27062F10E0E114F10471F081EE0E9495
:1036B000B206C801009741F0EFE9FFE03197F1F75A
:1036C00000C000000197F6CFC114D10439F44801BD
:1036D000B8018B2D0E942F07C8010EC086EE0E94F4
:1036E000B206C801009799F3EFE9FFE03197F1F7CF
:1036F00000C000000197F6CF009741F0EFE9FFE02E
:103700003197F1F700C000000197F6CFCD2819F5E9
:10371000EF2879F081EE0E94FC060115110549F0B1
:103720008FE99FE00197F1F700C0000001501109F7
:10373000F4CFCD2BF1F08CE20E9447078114910465
:10374000C1F0EFE9FFE03197F1F700C00000F1E0D0
:103750008F1A9108F3CF86EE0E94FC06C8010097ED
:10376000B9F2EFE9FFE03197F1F700C000000197EF
:10377000F6CFDF91CF911F910F91FF90EF90DF90E7
:10378000CF90BF909F908F900895EF92FF920F93EC
:103790001F93CF93DF93EC01162F0AE088818823D3
:1037A00009F457C0813009F04FC08981813041F45C
:1037B0007E0182E0E80EF11C8A810E94470709C061
:1037C000823049F47E01E2E0EE0EF11C8A810E9413
:1037D000B206E7012DC0833041F47E01F2E0EF0E26
:1037E000F11C8A810E94FC06F4CF843011F02196EE
:1037F0001FC02A81229680E090E030E020533109FA
:103800002A30310558F4089FA001099F500D11245A
:10381000C901840F951F21962881EFCF009741F0B1
:10382000EFE9FFE03197F1F700C000000197F6CF14
:10383000812F90E0009759F0EFE9FFE03197F1F721
:1038400000C000000197F6CF612F0E94131B219644
:10385000A5CFCDB7DEB7E6E00C949C240F931F9361
:10386000CF93DF93C42FD22FFC0185818823B1F041
:1038700040935C020E94702090935B0280935A02F6
:1038800080E28C0F883008F04DC0C77081E001C025
:10389000880FCA95EAF70E94510744C080915C02E4
:1038A000481330C080915A0290915B020E94882098
:1038B000883C910538F510E21D0FCD17B9F080E274
:1038C0008C0F883040F4C77081E001C0880FCA9522
:1038D000EAF70E945807183010F581E09D2F977085
:1038E00001C0880F9A95EAF70E945107802F0E9425
:1038F00047071830B8F4D77081E001C0880FDA9517
:10390000EAF70AC080E28C0F883060F4C77081E06B
:1039100001C0880FCA95EAF70E94580703C0802F9C
:103920000E944707DF91CF911F910F9108950F9348
:10393000FC01E851FC47E730F10590F5CB01EE5969
:10394000FF4F0C94672406E221EE41EE6AE17CE72A
:1039500023C007E225EE45EE6BE17CE71DC006E2E1
:1039600021EE40EE68E17CE717C007E225EE44EE69
:1039700069E17CE711C006E221EE42EE6CE17CE7F2
:103980000BC007E225EE46EE6DE17CE705C008E2DC
:1039900021E045EE6EE17CE70E942E1C80E008C02D
:1039A000FB018581882319F010925C0201C081E03F
:1039B0000F9108951F93CF93DF9387372CE79207DA
:1039C00021F088379C4759F031C0FB01C581CC23D9
:1039D00019F00E941C1D09C00E941C1D18C0FB018B
:1039E000C581CC2391F00E941F1D0E941A0A0E94DB
:1039F000221DD82F0E941F1DC82F0E941C1D4D2F55
:103A00006C2F0E94440BC0E012C00E941F1D0E9438
:103A1000260A0E94221D182F0E941F1DD82F0E94C7
:103A20001C1D412F6D2F0E94440B01C0C1E08C2F43
:103A3000DF91CF911F91089580910C01089580919D
:103A40000B01089580910A01089584E290E00E949C
:103A5000D524853281F485E290E00E94D52481301E
:103A600051F486E290E00E94D52491E0843109F07F
:103A700090E0892F01C080E081700895CF93C82F16
:103A8000811102C06FEF01C065E284E290E00E9404
:103A9000F324C11102C06FEF01C061E085E290E044
:103AA0000E94F324C11102C06FEF01C064E186E2FD
:103AB00090E00E94F324CF9108950895CF92DF9271
:103AC000EF92FF92CF93DF93C7E2D0E060E070E027
:103AD000CB01CC24D62EE72EF82ECE010E94D52481
:103AE000A7019601282BCA01B9012196CA32D10536
:103AF00081F7DF91CF91FF90EF90DF90CF90089505
:103B00000895CF92DF92EF92FF926B017C010E94A9
:103B1000801D6C2D89E290E00E94F32499278F2D5F
:103B20007E2D6D2D88E290E00E94F324B701882756
:103B3000992787E290E00E94F324FF90EF90DF90B6
:103B4000CF90089580E00E943E1D60E070E0CB01C0
:103B50000E94811D0E9430160E94E51681E00E949D
:103B60003E1D08950E945D1D0E945E1D0E94801DE5
:103B70000E94251D811102C00E94A21D0895089572
:103B80009C01FB018581882351F0A90157574038DA
:103B9000510530F4C9010E94F51680E0089581E0D6
:103BA00008952FEFFC01208308950E94D11D0895F0
:103BB00080E00895A0E0B0E0E0EEFDE10C947C240C
:103BC000EC01F62E0E94D81D8111BEC0E8818E2F17
:103BD00090E0FC013197E331F10508F0AFC0E759FF
:103BE000FF4F0C94672419828CE06BC0898182306E
:103BF00089F030F4813009F0A1C00E947C200CC013
:103C0000833079F0843009F099C01A821B821C82BB
:103C10001D8296C00E945E1D9A838B837C836D8378
:103C20008FC0EA806E0183E0C80ED11C00E010E076
:103C3000AE2CB12CC501800F911F0B9708F080C0EE
:103C40008E2D800F0E94FE12F60181936F010F5F8F
:103C50001F4F0C31110571F773C08981823039F023
:103C6000853009F06BC08A810E94BF1D69C06A81DE
:103C70007B818C819D810E946D240E94811D60C08A
:103C80004B816A8189810E94F4159C838D8358C081
:103C90002C813D813227232732274B816A818981FC
:103CA0000E9415164DC00E9430164AC06F2DCE01DD
:103CB0000E94D51D45C00E949C1624C00E949E16DD
:103CC00099838A833DC06B8170E089819A81AE01BE
:103CD0004C5F5F4F9827892798270E94A11630C014
:103CE0006B8170E089819A81AE014C5F5F4F9827AC
:103CF000892798270E94C41623C00E94E51620C079
:103D00000E94E11589831CC06B8170E089819A81D2
:103D1000AE014C5F5F4F9827892798270E944E1667
:103D20000FC06B8170E089819A81AE014C5F5F4F5B
:103D30009827892798270E94701602C08FEF8883E2
:103D40006F2DCE010E94F121CDB7DEB7EAE00C94D1
:103D5000982490936202809361020895E091610239
:103D6000F0916202309729F00190F081E02D0995E1
:103D7000089580E00895E0916102F0916202309729
:103D800021F00280F381E02D09950895E091610210
:103D9000F0916202309739F022E0DC012C9306802A
:103DA000F781E02D09950895A3E0B0E0EAEDFEE18A
:103DB0000C94842420915F02309160022817390707
:103DC000A1F09093600280935F02E0916102F09114
:103DD0006202309751F023E029839B838A83008419
:103DE000F185E02DCE01019609952396E2E00C9431
:103DF000A024A3E0B0E0EFEFFEE10C948424209136
:103E00005D0230915E0228173907A1F090935E029F
:103E100080935D02E0916102F0916202309751F06F
:103E200024E029839B838A830084F185E02DCE01E1
:103E3000019609952396E2E00C94A024E0910001FC
:103E4000F0910101329697E080E0915029F02191A4
:103E50002223D9F38F5FF9CF0895882371F0209141
:103E6000000130910101F9013296285F3F4F919195
:103E7000891729F0E217F307D1F780E0089581E070
